:020000020000FC
:100000005ACEBBC10000000020C000008DC000001F
:10001000000097C00000000000000000020304067A
:10002000080C10182030406080000406080C1018DE
:100030002030406080A0C0000003070F1F000D0D9E
:100040000403060D0503030202004FB662FD0CC057
:10005000552041F00994C52DC095089483FDC7959E
:10006000C4BD64604FBE1895C0916400089483FDC0
:10007000C795C4BD6B7FC0916400CF3F09F41DC01C
:1000800070FF19C082FD05C04FBEC098AC9895980E
:100090001895C098AC98959876FD0DC065FD0BC07D
:1000A000C9E0CA95F1F7C091B100C0FDAB9AC1FD9E
:1000B000AD9AC2FD949A4FBE189524BCCC27C0645B
:1000C000C8BF6460F8CFC7CF70FFC5CF65FDC3CF91
:1000D000C09AC1CF70FFBFCF65FDBDCFAC9ABBCF7B
:1000E00070FFB9CF65FDB7CF959AB5CFAB9870FFCC
:1000F000B2CF65FDB0CFC7E0CA95F1F7C09AABCFDC
:10010000AD9870FFA8CF65FDA6CFC7E0CA95F1F7FF
:10011000AC9AA1CF949870FF9ECF65FD9CCFC7E0AD
:10012000CA95F1F7959A97CF4FB6C9B7CF7EC9BF99
:100130006E7FCCB5CE0DDDB5DF1DDBBDCABD4FBEBC
:1001400018953FB68F7EABB7A074A2118061A0E076
:10015000ABBFA9B7AE7FA9BF7894A0916800AA23CE
:1001600041F085FD2AC0A0916800AA95A09368007F
:1001700024C040E050E085FD14C0A0B396FDA095DA
:10018000A2FD4FEFA3E096FDA2E0A5BFAA27A064C1
:10019000AABF8D7FA0B396FDA095A2FD5FEF451786
:1001A00041F7A0E461FDA093680085FD03C0A0E4D1
:1001B000A093680040939600816085FD0EC0A091D9
:1001C0006900AA2331F0A0916900AA95A093690063
:1001D00004C08061AA27A064AABF80FF0AC0A091C2
:1001E00096004A2F61FF8E7F85FD01C000C04093BD
:1001F00061004091B400443009F004C0A091610056
:10020000A0936300A52DA03408F06860A091600061
:10021000A395A093600051F0F894A9B7A160A9BF7D
:1002200084FF02C0A0E4ABBF3FBE1895A09174004C
:10023000A395A093740042E050916800552329F0E3
:1002400085FF03C05A9550936800A0919600A13095
:1002500018F0209299000DC020929A002092A300DD
:10026000A0919900AF5FA093990018F0AFEFA09311
:100270009900B09061005091B400523049F466FF8B
:1002800091F0A2E3BA1678F0A0918600A0936100E5
:10029000533049F466FF39F0A2E3BA1620F0A0917A
:1002A000C000A0936100509162005B1521F010F036
:1002B0005A9501C05395509362004A95D1F65091DA
:1002C000A300539509F45A955093A300A091A4005C
:1002D000AA95A093A40009F046C0A1E0A093A400B1
:1002E00045E0A091A5005A17F0F1A091A6005A1779
:1002F00028F441E0A3E0A093A40007C0A091A700C8
:100300005A1718F441E04093A400D0909C00C0908C
:100310006300DC14A8F0A091B400A430D9F066FD0D
:100320000FC0C0929C00539511F0A091A500A0931E
:10033000A300A1E0A093A400ACE3A093620013C0CB
:10034000A0919C00A40F20F45FEF50939C0002C08A
:10035000A0939C00A0919C00AF3F29F4AFEFA09325
:100360009A00A093A300F894A9B7A160A9BF84FF45
:1003700002C0A0E4ABBF3FBE18953FB64CB55DB51B
:100380008F7EABB7A074A2118061A0E0ABBFA9B70C
:10039000AE7FA9BF789481FD23C0A2E096FDA3E0C3
:1003A000A5BF8260A0B396FDA095A2FF05C04093B3
:1003B0006500509366001CC1A3E096FDA2E0A5BFB6
:1003C000AA27A064AABF8D7F85FF01C004C140E0B9
:1003D000A0B396FDA095A2FDFEC040939600EDC08F
:1003E000A3E096FDA2E0A5BF8D7F61FF71C0A2E0F2
:1003F00096FDA3E0A5BFAA27A064AABF8260409390
:10040000910050939200A0908F004A19B0909000F4
:100410005B09BB24A22C4C38520518F4209295009D
:1004200049C0A091D400AA2359F1483C520528F4B0
:10043000A0E1BA2EAAE0AA2E23C04836A1E05A07AE
:1004400028F4A8E0BA2EAFE0AA2E1AC0403DA2E0E0
:100450005A0728F4A4E0BA2EAEE1AA2E11C0403A01
:10046000A5E05A0728F4A2E0BA2EACE3AA2E08C0F1
:100470004839A8E05A0720F4A1E0BA2EA8E7AA2E2E
:10048000C42EA0919300CA1AD52EA0919400DA0A26
:10049000DD202AF4AFEFC094D094CA1ADA0A209271
:1004A0009500A8E0A210A0E0CA14DA0618F4A1E0B2
:1004B000A093950040939300509394004091910035
:1004C0005091920040938F005093900042E075C08D
:1004D000A09165004A1BA09166005A0B94FD60C074
:1004E00093FD5EC092FD5AC086FF03C0D52EC42E78
:1004F0000CC05695479591FD51C05695479590FD76
:100500004DC0D52EC42ED694C79461FD19C0AC2D14
:10051000AC51AD2DA24008F005C0DD2089F4AC2D12
:10052000A85C70F4A0916700A395AA2311F0A09392
:100530006700AA3008F44FC02092960081604BC03B
:10054000A0916700AA2319F0AA95A0936700A22C96
:100550005091BA0097FD02C0A090C800AAEFAA0E61
:10056000A22DA21DCA18DA0A4FB74170442319F010
:1005700040E050E015C0AFEFCA16D20418F04FEFBC
:1005800050E00EC0A091AC00CA9E412D000C441F4B
:1005900050E008F012C04FEF50E00FC0569547955D
:1005A00094FF07C0552309F04FEFA42FA6954A0FDB
:1005B000521D4F3F520508F04FEF40939600816067
:1005C00061FF09C0AFE1A095A923AB299A2F8F7DC8
:1005D000BB2009F48062A0E4A093680085FF03C0FB
:1005E000AAE0A093680061FD03C085FD01C08F7E75
:1005F00085FD03C0A0E2A0936900F894A9B7A160AB
:10060000A9BF84FF02C0A0E4ABBF3FBE189511E0B4
:100610000AC013E008C01AE006C01EE104C014E6D8
:1006200002C018EC00C005E1BB27BA95F1F70A95A6
:10063000D9F71A95C1F708952AE338E709C020E3EE
:100640003CE806C02AE234EB03C025E238EC00C0E7
:1006500012E0BB27AD98BA95F1F7AC9ABA95F1F7CD
:10066000AC98BA95F1F7AD9ABA95F1F7123009F056
:10067000C09A123009F4959AB091AD00BA95F1F78D
:10068000123009F0C098123009F49598B7E8BA957D
:10069000F1F71A95F1F6022FB22FBA95F1F70A95F4
:1006A000D9F73A95A9F6AD980895221B39E0001FB5
:1006B0003A9509F40895221F211B18F4210F8894FC
:1006C000F6CF0894F4CF622C722CB0E08894B395E6
:1006D000221F331FE0F7379527958894912E802E9F
:1006E000020B130B10F4192D082D10F4889401C07F
:1006F0000894661C771CBA9571F7172D062D08957E
:10070000322D11232AF43A9500951095031B130BF3
:10071000F894029F712C002D129F912C802C7894BC
:10072000780C172D921C292DB4E06B2E2695179569
:1007300007956A94D9F7332321F000951095031B90
:10074000130B08950091B400043009F474C0B09103
:100750009600B95198F0B72FB67081F466FD2BC0A2
:1007600005E09090C600B92DBA9521F00AE0BA953F
:1007700009F002E1B0917B00B01BE0F066FF0AC017
:10078000B0919E00B0939C00BFEFB093A300B1E086
:10079000B093A400B0916100B093630020927E00FA
:1007A00020927F002092800020928100209282007F
:1007B0006F7B41C060649090C600B92DBA9579F402
:1007C000B0916200B095BB1FBB1F1B2FB7950B2FBD
:1007D000B12FB170B3951B2FB02FBE7F25C0B92D9F
:1007E000BA95BA9581F4B0916200B095BB1FBB1F5A
:1007F000BB1F1B2FB7950B2FB12FB370B3951B2FBA
:10080000B02FBC7F14C0B0916200B095BB1FBB1F5E
:10081000BB1FBB1F1B2FB7950B2FB12FB770B39505
:10082000B3951B2FB02FB87FB0540B2F1209009334
:100830007E0010937F00089510917B001695009123
:100840007A000795B0917E00B01B0B2FB0917F000E
:10085000B10B1B2F28F40038BFEF1B0740F009C075
:100860000F37120508F405C00FE710E002C000E8DA
:100870001FEF00938300109384000895009183007C
:10088000B09180000B0F10918400B09181001B1F6C
:1008900020E03091840033230AF42A95B09182003D
:1008A0002B1F1AF4203F40F00AC02F3008F407C075
:1008B0000FEF1FEF2FE003C000E010E020EF3091BA
:1008C0006300B0919B003B1718F4323030F009C040
:1008D000B0918400BB235AF004C0B0918400BB23C4
:1008E00032F40093800010938100209382000895D9
:1008F0002091D70000918300000F10918400111FF8
:10090000FFDE11232AF40038BFEF1B0740F009C0B7
:100910000F37120508F405C00FE710E002C000E829
:100920001FEF002352F0B0916200B01B0B2F18F0A4
:10093000013008F00AC001E008C000950F5FB091D7
:1009400062000B0F08F001C00FEF009385000895BF
:100950002091D8000091810010918200D1DE1123F6
:100960002AF40130BFEF1B0740F009C00F3F12050A
:1009700008F405C00FEF10E002C001E01FEF1123E3
:1009800052F0B0918500B01B0B2F18F0013008F029
:100990000AC001E008C000950F5FB09185000B0F01
:1009A00008F001C00FEF0093630008950FEF677F19
:1009B00071FD29C072FD09C06860B0917B00BA303A
:1009C00020F0B52DB03408F4677FB091D300BB237D
:1009D000D1F0B0917B00BB23B1F00FEF10917B0001
:1009E00064DEF894B091730072FDB5E00B9F112D99
:1009F000002D7894112309F00FEFB0919E000B1792
:100A000010F400919E0000939D00089500917A00DB
:100A100010917B0000541140B0919D0010F4BA95E4
:100A200001C0B39511F0B0939D000895E6D3B2E0F4
:100A300074FDB1E0B7B9B6B1B068B064B6B9E7DD7E
:100A4000B2E074FDB1E0B7B9B6B1B068B064B6B9A0
:100A5000B6B1B6FDFDCF04B115B1B6B1BF77B6B929
:100A600025D424E72093A800222309F441C030E0D4
:100A70003093A900732E7694622E6694620E731ED4
:100A8000262D372D0217130778F08090A800B4E7C1
:100A9000B80DB093A8008090A900B0E0B81DB09345
:100AA000A900260D371DEECF8090A8009090A900D8
:100AB0001091A90016950091A80007951695079525
:100AC00023E0169507952A95E1F72091B5002A9520
:100AD00029F42092A8002092A9000AC02A9521F0AA
:100AE000800E911E2A95E1F78092A8009092A900AD
:100AF00008952091B500B6B1B6FDFBCF04B115B194
:100B0000B6B1BF77B6B9B091AA00B395B093AA00B9
:100B1000B83060F12092AA00B091D200BB2321F13D
:100B2000112329F0B091AB00BF3F61F009C0B09133
:100B3000AB000B1739F020F4BB2321F0BA9502C0AB
:100B4000B395E1F300919B00B093AB00B13A50F440
:100B500000ECB43938F400E8B73820F400E4BA37D0
:100B600008F400E000939B007F7E08952130B1F0EF
:100B70000F3FB3E01B0790F4B4E7BB2379F0B091CB
:100B8000A8000B17B091A9001B0740F4B0919B007F
:100B9000BB2359F0BA95B0939B0007C0B0919B005E
:100BA000BF3F19F0B395B0939B0000919B00B091AB
:100BB0006300B01B10F400916300B0919C000B1710
:100BC00050F000919C00B0919C00BF3F21F0B0918B
:100BD0009C00B0939B00502E00936400B091AA003B
:100BE000B73009F47061089502E3F894B091D90028
:100BF0000B9F012D000C001F7894B0919B000B17E8
:100C000010F000919B000093610000936300502E50
:100C10000093640000939E00089520927A00B0EF44
:100C2000B0937B000895F8940CB51DB52091740025
:100C30007894309175006090760000937500109361
:100C40007600031B160971FD03C077FD7DC027C028
:100C500070907700209377002709222311F00FEF7F
:100C60001FEF809078009090790030937800609228
:100C700079000091750010917600081919092091EA
:100C80007A0030917B0036952795020F131F10F4E0
:100C90000FEF1FEF00937A0010937B0029C0209183
:100CA0007A0030917B003901B4E08B2EB2E09B2EAC
:100CB000343010F08A949A94383010F08A949A94D0
:100CC000769467948A94E1F726193709992021F0E0
:100CD000169507959A94E1F7200F311F20937A001B
:100CE00030937B0028F43FEF30937A0030937B0001
:100CF000323008F4706871FF02C0B3E00DC0B091EB
:100D0000C40000917100023838F0B395003A08F041
:100D1000B395B63008F0B5E09B2EB4E08B2E109161
:100D20007B0000917A0024E0169507952A95E1F75B
:100D30000819120928F0B02FB250B12FB20910F4DF
:100D400002E010E0980126C020917A0030917B00EB
:100D500039017694679466946694669426193209EC
:100D600006950695200F321D20937A0030937B0064
:100D7000323008F07F7704E0369527953695279531
:100D800026952695201B10F0223008F422E08901D8
:100D90009090C40060FDFECFE0908B00F0908C003E
:100DA0006160B9B7B061B9BF380177FD41C07694D1
:100DB000679400938B0010938C00B92DB330E1F051
:100DC000B0FD04C0060D171D930106C0000F111FD2
:100DD0000250120922E030E0B92DB33068F02093C0
:100DE0008D0030938E0000938700109388006092EE
:100DF000890070928A003AC000938D0010938E0093
:100E000020938700309388006092890070928A0056
:100E100071FF0DC0BFE0B0938D0020928E00B093A3
:100E2000890020928A00B0938B0020928C001EC013
:100E3000669400938B00B92DB33091F0B0FD03C0E0
:100E4000060D262D03C0000F025022E0B92DB3304D
:100E500038F020938D00009387006092890006C0CF
:100E600000938D00209387006092890000917C00A0
:100E700002FD0350013029F495FD0AC0B0E0B7B976
:100E800009C0023019F4B7E0B7B904C095FDF6CF38
:100E9000B6E0B7B90091A200000F10F4BBE60B2733
:100EA0000093A20060FDFECFB2E0B0936E006160DF
:100EB000B9B7B061B9BFB72FB670D1F020917A0041
:100EC00030917B00369527953695279571FF02C0A6
:100ED000B0E43B0FF8940CB51DB5020F131F1BBDFA
:100EE0000ABD6160B0E1B8BFB9B7B061B9BF78946D
:100EF0000895606120927D0020E067FD20E206C039
:100F0000606120927D0020E267FD20E001E011E0B9
:100F100077FD11C0B72FB67009F06F7E14E1009114
:100F20007B00069509F403950F3008F00FE071FF80
:100F300002C004E114E160FD0FC0B0917D00BB234D
:100F400059F071FF06C0B0916E00BA95B0936E0073
:100F500011F4706247C0ABDFB0B7B77FB0BFB8B1B4
:100F6000B0B7B860B0BFB0917D00B395B0937D00CD
:100F7000B8B177FD06C0B1E071FDB3E0BA95F1F705
:100F8000B8B1B072B21709F022C071FF05C0039565
:100F9000011708F00A95CFCF64FD05C0039501172E
:100FA00008F0B4CFC8CF6F7EF8943CB56DB47090A4
:100FB0007A0080907B00370D681C6BBC3ABD616085
:100FC000B0E1B8BFB9B7B061B9BF78949FCFB09165
:100FD0006D00B13008F49ACF64FD98CF0A9509F0FE
:100FE000AACF7F7D20918D0030918E00F894B0E1E2
:100FF000B8BF0CB51DB5020F131F1BBD0ABDE09095
:101000008700F09088006160B9B7B061B9BF78948B
:10101000B72FB67039F0B0916D0072FFB395B093F1
:101020006D0009C075FF07C067FD05C064FD03C002
:10103000BF91BF91EBC4089500E063FF03C064FF5C
:1010400001C001E0F89410917100B7E01B9F212DC1
:10105000102D7894200F269517952695179526958F
:10106000179510937100183718F4B8E7B093710012
:1010700000917100B09172000B1720F06062C0986F
:10108000AC98959860FDFECFE0908900F0908A00C2
:101090006160B9B7B061B9BF0895C49AB2E095FD77
:1010A0000AC0F894B0937C00AD98AB9A62FF01C07F
:1010B000959A7894F9C0F894B0937C00AD98949A7E
:1010C00062FF01C0C09A7894EFC0C498B3E082FF79
:1010D00024C095FD11C002E0F894B0937C00E0E8D4
:1010E000F0E00093B1009598949862FF02C0AC9A2A
:1010F00001C0AD9A7894D8C002E0F894B0937C0017
:10110000E0E8F0E00093B100C098AB9862FF02C045
:10111000AC9A01C0AD9A7894C7C095FD0BC0F89405
:10112000B0937C00EAE6F0E0959862FF01C0AC9ACB
:101130007894BAC0F894B0937C00EAE6F0E0C098E6
:1011400062FF01C0AC9A7894AFC0C49AB4E095FD38
:101150000AC0F894B0937C00AB98949A62FF01C0E7
:10116000AC9A7894A1C0F894B0937C009498AB9A10
:1011700062FF01C0AC9A789497C0C498B5E082FF32
:1011800024C095FD11C001E0F894B0937C00E6E71F
:10119000F0E00093B100AC98AD9862FF02C0C09A35
:1011A00001C0AB9A789480C004E0F894B0937C00BE
:1011B000EAE8F0E00093B100AC98AD9862FF02C09D
:1011C000959A01C0949A78946FC095FD0BC0F894DD
:1011D000B0937C00E4E6F0E0AC9862FF01C0C09AF6
:1011E000789462C0F894B0937C00E0E7F0E0AC98AB
:1011F00062FF01C0959A789457C0C49AB6E095FDF5
:101200000AC0F894B0937C009498AD9A62FF01C034
:10121000C09A789449C0F894B0937C00AB98AD9A8A
:1012200062FF01C0959A78943FC0C498B1E082FFF4
:1012300024C095FD11C004E0F894B0937C00EAE866
:10124000F0E00093B100C098AB9862FF02C0959A9D
:1012500001C0949A789428C001E0F894B0937C007F
:10126000E6E7F0E00093B1009598949862FF02C021
:10127000C09A01C0AB9A789417C095FD0BC0F89442
:10128000B0937C00E0E7F0E0C09862FF01C0959A5F
:1012900078940AC0F894B0937C00E4E6F0E0959866
:1012A00062FF01C0C09A78946F7D089523E630E014
:1012B000F9012092B100C098AC989598AB98AD9880
:1012C00094986B7F0895A2EBB0E007E00D9307E0E0
:1012D0000D9301E00D9304E00D930FEF0D930D932B
:1012E00009E00D9302E00D9301E00D9301E00D93F1
:1012F000AEEBB0E001E00D9300E00D9304EB0D9335
:101300000FEF0D930D930D9303E00D930FEF0D93DE
:1013100001E00D930FEF0D9305E20D9300ED0D939A
:1013200008E70D9308EC0D9304E00D930FEF0D9378
:1013300001E00D9300E00D930AE70D930AE00D9391
:1013400000E00D9301E00D9300E00D930FEF0D937E
:1013500000E00D9308952091B9008B7F233009F4AC
:101360008460B091BA009F7DB1FD90629F7BB09187
:10137000BB00B1FD9064223011F0886001C0877F0E
:1013800008950A95E00FF21DB4910895ECE1F0E0A4
:101390000091B200F6DFB093D700ECE1F0E00091ED
:1013A000B300EFDFB093D800EAE2F0E00091B800BC
:1013B000E8DFB093D9000091D100002309F4039530
:1013C000013108F001E1B02FB00FB00FB093A500CC
:1013D0001B2FB10FB10FB00FB093A600B10FB00F1C
:1013E000B00FB093A7000091B800023008F402E0FB
:1013F00000937300B091CE000FEFB23009F400EA11
:10140000B33009F402E800937200E8E3F0E00091E1
:10141000D500B7DFB093A000089508952091C800CB
:101420003091C900B091BA00B33009F43E5097FF33
:1014300002C020E03FEFB32FB21B6B2EB25810F466
:10144000B2E86B2E00E00395609EB12DBD57D8F336
:101450000093AC0008959068E1DFDFD820E030E031
:10146000B0E16B2ED6D8B09196002B0F321D6A9446
:10147000C9F7B4E036952795BA95E1F7822E9F77A4
:10148000CDDF0895F894E3E0F0E0B9E0B7BFB491A0
:10149000B078C1F3F894A895B1B5B861B1BDB0E02A
:1014A000B1BDB4E0BEBFBFE5BDBF00DFB0E0B8BBBB
:1014B000B1E1B7BBB0E0B5BBB8E3B4BBB0E0B2BB21
:1014C000B0E3B1BB2224A0E0B0E02D92AA31E9F74D
:1014D000A0E6B0E00FEF2D920A95E9F7B1E0B093E6
:1014E000A200F1DED0D2B6B1B460B6B90091CA00A4
:1014F0000093AD00B1E0B0936A00F89492D89CD804
:101500008CD89DD88AD89ED888D84CD38AD889D8E8
:1015100086D8F8940AEF1AEFA0B396FDA095A2FF23
:101520001FC01A95C9F70A95B1F7E0E0FCE1B59143
:10153000B43E39F4B591B03E21F4B591BF3F09F402
:101540000CC0E0E0F395F395B591B83F49F4B5913F
:10155000B43931F4B591BA3A19F4EE27F6950994F5
:10156000FADE14DF5ADF5ADF0091CA000093AD00A3
:101570009DDEB2E0B3BFB2E0BEBDB2E0B5BDB1E545
:10158000B8BFB9BFB0B7B77FB0BFB8B1B0B7B86078
:10159000B0BF3DD878944ADA20927000B3E096FD4F
:1015A000B2E0B5BFB0E4BBBFBB27B064BABF8D7FAC
:1015B00038D8626033E02CE0B0919500BB2321F471
:1015C0002CE03A9509F4A5CF28D880FFA2CF8E7FD2
:1015D000B0919600B23078F3B92FBF7100919800A6
:1015E00000939700B0939800B01729F72A9521F738
:1015F0006D7FB3E096FDB2E0B5BFBB27B064BABF64
:101600008D7FB091D400BB2321F48062B92FB070DC
:101610009B2F8F7B2092670002D885FF05C0B09179
:101620006700BA3008F08064F4D702E085FF01C09B
:1016300000E0B0919600B017B8F3F894FDD7FCD74E
:10164000FBD77894EED720928600E3D7B091BE0006
:10165000B13008F46EC0B0916A00B13008F469C0CE
:1016600085FD18C0B0919600BF3F08F462C0F894A1
:10167000ECD77894D4D7B0919600B130C0F7F894F5
:10168000DBD7C9D7D9D77894CAD7B0919600BF3FD6
:10169000B0F3BAC2B8E09B2E9068F894BFDE78949D
:1016A000BED7F8949F77BADE80909600B0919600EE
:1016B000BF37789408F445C0AAD7F894C6D7789471
:1016C0009A9451F7C8DEB82DB550B093C900A9D788
:1016D000F89406D26CD27894BAE09B2E9068F89475
:1016E0009DDE78949CD7F8949F7798DE8090960042
:1016F000B0919600BF37789478F789D7F8949CD743
:101700008AD79AD778949A9449F7A5DEB82DBB5F0B
:10171000B093C80086D7F894E3D158D278947FD795
:10172000F8947CDE7894B0919600BF3F08F498CF8F
:101730006BC200919600B09186000B1710F00093D9
:1017400086006DD701E0B091BA00B35009F405E00E
:10175000B0919600B01708F078CFF89476D775D787
:1017600074D778945ED720926A0020926B00209202
:101770006C00B0916B00B395B0936B00BF3F71F5F7
:10178000B0916C00B395B0936C00B091CC0009E1BE
:10179000BA9559F002E3BA9541F00DE7BA9529F0F0
:1017A0000AEFBA9511F020926C00B0916C00B0175E
:1017B000A8F07CDD2CD7B0916C00BA95B0936C008A
:1017C00020926B00B091CB00B093AD00F8943DD760
:1017D0007894B091CA00B093AD0021D71CD7B091D6
:1017E0006800BB2319F485FF01C093CE01E085FD9D
:1017F00001C006E0B0919600B01708F4BACF0FD739
:10180000B0916800BB2309F484CEF8944FDD209298
:1018100061002092620020926300522C20926400AA
:101820002092A1007894B091B700BB0FB0939F00B5
:1018300020927E0020927F002092800020928100E2
:10184000209282002092AA0060E070E02092710055
:10185000B8E0B093AA007061DAD6B2E074FDB1E0EE
:10186000B7B9B6B1B068B064B6B9B6B1B6FDFDCF20
:1018700004B115B1B6B1BF77B6B9112309F00FEFB6
:101880000093AB0036D9B8E0B093AA00706163DD75
:10189000F894BFEFB0939B00A7D9B0916100B093CB
:1018A0009B00B0939C00B0939D007894B1E0B093FE
:1018B0006100B09363005B2EB0936400B093A4000A
:1018C000B0919A00B093A300B091BA00B33019F46C
:1018D0009F7D87FD90627160726020926D008DDC4B
:1018E000A4DC9BD9A0D999D99ED997D909DB2AD74D
:1018F000A3DBD3DB98D9FDDA66FD9ED777FF56D8F8
:1019000077FD84D899DBE1DB8ED9FADA66FDB6D7AC
:1019100093DB1BDC88D9EDDA66FDEAD78DDB2DDCA5
:1019200082D9EEDA66FD14D887DB67DC7CD9E1DA90
:10193000B2E074FDB1E0B7B9B6B1B068B064B6B9A1
:101940007BDB73DC70D9D5D871FF1EC0B0919E00CF
:10195000B0939B00B0939C00B0919A00B093A30009
:10196000B1E0B093A40018E12CE0B0916D00B11784
:1019700028F07D7F746020936F0006C0B0919600C0
:10198000B13008F0B3CF4CC072FF11C067FD0FC07B
:10199000B0916F00BA9519F47B7F7860A7CFB093B0
:1019A0006F00B0919600B13008F0A0CF39C02092FE
:1019B0007000B0919900B13058F0B0919E00B09392
:1019C0009C00B0919A00B093A300B1E0B093A40042
:1019D000B09199000AEF1091D600112309F003E0AD
:1019E000B01708F01DC085FF04C0B0916800BB238C
:1019F000B9F000EF67FF05C0B0919E00B0939B0067
:101A000000E2B0917B00B01708F470CFB091700085
:101A1000B395B0937000B0919600BB2309F002C05B
:101A200020927000F89442DC8090B900B2E0B0934C
:101A3000B90091DC8092B90020926100209262008E
:101A400020926300522C2092640020929F0060E05C
:101A500070E07894E4D52ADC0091D600002319F0D8
:101A6000C09AAC9A959AB6B1B460B6B985FF05C074
:101A7000B0916800BB2309F44CCDB091BF00B130E8
:101A800008F0D2CD72CEEDE0F0E023D0053A09F0B7
:101A90001BC0EEE0F0E01DD00A3509F015C03AE0B9
:101AA000A2EBB0E0E3E0F0E014D00D9331963A956C
:101AB000D9F739E1AEEBB0E0EFE0F0E00AD00D93FA
:101AC00031963A95D9F702C0FEDB0AD0E8E2F0E0A1
:101AD0000895E199FECFEEBBFFBBE09A0DB30895E8
:101AE0001ED03AE0A2EBB0E0E3E0F0E00D910FD0C1
:101AF00031963A95D9F739E1AEEBB0E0EFE0F0E09E
:101B00000D9105D031963A95D9F712D00895E19903
:101B1000FECF0DBBEEBBFFBBE29AE19A0895EDE06C
:101B2000F0E00FEFF4DFEEE0F0E00FEFF0DF08950C
:101B3000EDE0F0E005EAEBDFEEE0F0E00AE5E7DFFC
:101B400008953091AE000091AF00313011F4009350
:101B5000B200323011F40093B300333011F400932B
:101B6000B400343011F40093C600353011F4009302
:101B7000B500363011F40093B800373011F40093FB
:101B8000C400383011F40093B900393011F40093D7
:101B9000CE003A3011F40093BA003B3011F40093B8
:101BA000BB00089525E03DD52A95E9F7089544D571
:101BB00046D548D54AD52FD53FD541D543D545D56E
:101BC0002AD53AD53CD53ED540D508953ED53AD50F
:101BD00036D532D520D539D535D531D52DD51BD5EE
:101BE00034D530D52CD528D508958090AE0090906E
:101BF000AF0022D521D520D50ED58A94D1F725D591
:101C00000AD59A94E1F70895F894D1DF7894CADF61
:101C1000C9DFB1E0B093AE00B1E0B093AF00209265
:101C2000B000F894E2DF7894B5E06B2E70909600E7
:101C3000F8D4B09196007B16C9F7B13018F0BF3FC9
:101C400040F107C07EDFF8944BDFB1DFB8E0B1BDF3
:101C5000A9DF6A9459F7B091B000B395B093B00082
:101C6000B33008F4DECF9EDFB091AF00B395B093F0
:101C7000AF00F894B091AE00BA95EEE3F0E0EB0F50
:101C8000F21D049178940395B091AF00B01708F459
:101C9000C6CF88DF87DFB091AE00B395B093AE00BA
:101CA000B091AE00BC3008F4B7CF0DDBF89418DF6C
:081CB000B8E0B1BD77DFE6CB1F
:00000001FF
